:100000000C9432000C944F000C944F000C944F0051
:100010000C94E0010C944F000C944F000C944F0092
:100020000C944F000C944F000C944F000C944F0014
:100030000C944F000C944F000C944F000C944F0004
:100040000C944F000C944F000C944F000C944F00F4
:100050000C944F000C944F000C944F000C944F00E4
:100060000C944F0011241FBECFEFD8E0DEBFCDBFF0
:1000700012E0A0E0B1E0E0E7FAE002C005900D92E6
:10008000A230B107D9F712E0A2E0B2E001C01D92A0
:10009000A730B107E1F70E9451000C9436050C948B
:1000A0000000AF92BF92CF92DF92EF92FF920F9338
:1000B0001F93DF93CF9300D00F92CDB7DEB780911F
:1000C000FEFF9091FFFF9B838A83A895809160003B
:1000D0008061877F80936000809360008FEF8093C2
:1000E0007E0083E080937F008FE18093640080B77F
:1000F000806880BF83B7817F83BF8FB78983F8947F
:1001000080E88093610081E08093610089818FBFE6
:10011000B090660080916400877F809364001092A5
:10012000700010926F008091B60088608093B600D6
:100130008091B60090E087709070892BC9F780E8B5
:10014000D82ECC24C394AA24AA941092B200109260
:10015000850010928400C092B000C0928100A7BABE
:10016000B89BFECF1092B000109281006091840085
:100170007091850080E090E00E947D027B018C01FF
:1001800020E83BEE42EF56E40E944D02882324F41F
:10019000809166008F5F0FC020E83CE545EF56E494
:1001A000C801B7010E941D02181614F081E006C0B4
:1001B0008091660081508093660080E0DA9419F0A7
:1001C000882319F204C0882311F4B092660080914C
:1001D000B600877F8093B60080916400886080932A
:1001E00064001092B000109270000E94D701892B19
:1001F00009F0FFCF8091B60088608093B6008091AF
:10020000B000887F8093B0008091B00081608093BF
:10021000B00080E00E94AB01F8941092640010924C
:100220007E0010927F0095B79C7F85B7816085BF67
:1002300095BFE0E0F0E0099580E090E00F900F902E
:100240000F90CF91DF911F910F91FF90EF90DF9072
:10025000CF90BF90AF900895FF920F931F939C0192
:1002600068EE73E00E94EB04082FF92EC90168EED6
:1002700073E00E94EB04FB0124E0EE0FFF1F2A95C0
:10028000E1F7802F9F2D64E670E00E94EB04482F79
:10029000192F802F9F2D64E670E00E94EB049B01D4
:1002A0002E0F3F1F94E0220F331F9A95E1F7842F02
:1002B000912F6AE070E00E94EB04260F371F84E064
:1002C000220F331F8A95E1F7842F912F6AE070E0A7
:1002D0000E94EB04282B392BC9011F910F91FF902D
:1002E0000895FC01EF70F070AC01452F5527429541
:1002F0004F7028EE33E0429FB001439F700D529F34
:10030000700D11246E0F7F1F9C01207F3070A4E0C0
:1003100036952795AA95E1F7A901F3E0440F551FFB
:10032000FA95E1F7220F331F420F531F640F751F19
:1003300080709F70892F992724E630E0AC01429F9E
:10034000C001439F900D529F900D1124680F791F9B
:10035000CB0108950895882319F0833039F510C032
:100360008091B00088678093B000809170008260B7
:100370008093700080EA8093B30010920202089587
:100380008091B00088678093B00080917000826097
:100390008093700080EA8093B30088E090E09093AF
:1003A00006028093050281E08093020208952F9A4D
:1003B000279A2F9A81E00E94AB0180E090E0089597
:1003C0001F920F920FB60F9211242F933F938F938A
:1003D0009F9380910202882339F1809103029091CA
:1003E0000402019790930402809303020196E1F4C2
:1003F0008091000190E021E030E0822793278093F4
:100400000001882321F48091B0008F7C03C080918B
:10041000B00080638093B000809105029091060245
:1004200090930402809303029F918F913F912F91AB
:100430000F900FBE0F901F901895A8E1B0E0E3E277
:10044000F2E00C940B0569837A838B839C832D8364
:100450003E834F83588789E0E82EF12CEC0EFD1E79
:10046000B701CE0101960E941A048E010F5E1F4F44
:10047000B801CE0105960E941A048985823040F0A9
:100480008989823028F0B801C7010E94920401C016
:100490008FEF6896E6E00C942705A8E1B0E0E3E56D
:1004A000F2E00C940B0569837A838B839C832D8304
:1004B0003E834F83588789E0E82EF12CEC0EFD1E19
:1004C000B701CE0101960E941A048E010F5E1F4FE4
:1004D000B801CE0105960E941A048985823040F049
:1004E0008989823028F0B801C7010E94920401C0B6
:1004F00081E06896E6E00C942705A8E0B0E0E3E828
:10050000F2E00C9409057B018C01611571058105F0
:10051000910519F482E0898360C083E089838EE1CC
:10052000C82ED12CDC82CB82ED82FE820F8318870D
:10053000C801B7010E94F602BC016150704077FF0C
:1005400039C0EE27FF27E61BF70B20E030E040E044
:1005500050E081E090E0A0E0B0E00E2E04C0880FF3
:10056000991FAA1FBB1F0A94D2F70197A109B109CD
:100570008E219F21A023B1230097A105B10521F071
:1005800021E030E040E050E004C016950795F79474
:10059000E794EA95D2F72E293F29402B512B2D8342
:1005A0003E834F8358878EE190E0861B970B9C8398
:1005B0008B8313C06115710581F0062E04C0EE0C0B
:1005C000FF1C001F111F0A94D2F7ED82FE820F83D9
:1005D0001887C61AD70ADC82CB821A82CE0101960E
:1005E0000E9445032896E8E00C942505EF92FF92BF
:1005F0000F931F937B018C0180E0E81680E0F806E2
:1006000081E0080780E0180788F48FEFE816F1040E
:100610000105110531F028F088E090E0A0E0B0E09D
:1006200017C080E090E0A0E0B0E012C080E0E816E3
:1006300080E0F80680E0080781E0180728F088E1EC
:1006400090E0A0E0B0E004C080E190E0A0E0B0E085
:1006500020E230E040E050E0281B390B4A0B5B0BF6
:1006600004C016950795F794E7948A95D2F7F70199
:10067000EF5FFE4F8081281B310941095109C901F3
:100680001F910F91FF90EF900895DF92EF92FF92EC
:100690000F931F93FC01E480F58006811781D180C0
:1006A0008081823048F480E090E0A0E1B0E0E82A68
:1006B000F92A0A2B1B2BA5C0843009F49FC0823075
:1006C00021F4EE24FF24870105C0E114F1040105A3
:1006D000110519F4E0E0F0E096C0628173819FEFAC
:1006E000623879070CF05BC022E83FEF261B370B1E
:1006F0002A3131052CF020E030E040E050E02AC003
:10070000B801A701022E04C07695679557954795C5
:100710000A94D2F781E090E0A0E0B0E004C0880F36
:10072000991FAA1FBB1F2A95D2F70197A109B109EA
:100730008E219F21A023B1230097A105B10521F0AF
:1007400081E090E0A0E0B0E09A01AB01282B392BCA
:100750004A2B5B2BDA01C9018F779070A070B070C3
:1007600080349105A105B10539F427FF09C0205C4B
:100770003F4F4F4F5F4F04C0215C3F4F4F4F5F4F84
:10078000E0E0F0E02030A0E03A07A0E04A07A0E473
:100790005A0710F0E1E0F0E079018A0127C06038E3
:1007A000710564F5FB01E158FF4FD801C7018F7750
:1007B0009070A070B07080349105A105B10539F436
:1007C000E7FE0DC080E490E0A0E0B0E004C08FE35D
:1007D00090E0A0E0B0E0E80EF91E0A1F1B1F17FF13
:1007E00005C016950795F794E794319687E016951E
:1007F0000795F794E7948A95D1F705C0EE24FF2476
:100800008701EFEFF0E06E2F679566276795902FD1
:100810009F77D794DD24D7948E2F8695492F462B2A
:10082000582F5D29B701CA011F910F91FF90EF90DA
:10083000DF900895FC01DB01408151812281622F0C
:100840006F7770E0221F2227221F9381892F880F44
:10085000822B282F30E0991F9927991F11969C937E
:10086000119721153105A9F541155105610571054E
:1008700011F482E037C082E89FEF13969C938E9329
:1008800012979A01AB0167E0220F331F441F551FD7
:100890006A95D1F783E08C930DC0220F331F441F5C
:1008A000551F12968D919C911397019713969C93C7
:1008B0008E931297203080E0380780E0480780E46C
:1008C000580758F314962D933D934D935C931797C7
:1008D00008952F3F310579F44115510561057105E2
:1008E00019F484E08C93089564FF03C081E08C9335
:1008F00012C01C9210C02F57304013963C932E9379
:10090000129783E08C9387E0440F551F661F771F73
:100910008A95D1F7706414964D935D936D937C9393
:10092000179708951F93DC01FB019C91923008F406
:1009300047C08081823008F443C0943051F411964E
:100940001C91843099F58181682F70E0611B7109D9
:100950003FC0843021F0923031F48230B9F181818E
:10096000882389F12DC011961C9111978230F1F0E6
:1009700081811817D9F412962D913C911397828199
:1009800093818217930794F028173907BCF01496C7
:100990008D919D910D90BC91A02D24813581468132
:1009A0005781281739074A075B0718F4112341F0CC
:1009B0000AC082179307A407B50740F4112319F062
:1009C00061E070E005C06FEF7FEF02C060E070E0B3
:1009D000CB011F910895AA1BBB1B51E107C0AA1FA1
:1009E000BB1FA617B70710F0A61BB70B881F991FD0
:1009F0005A95A9F780959095BC01CD0108952F9245
:100A00003F924F925F926F927F928F929F92AF929E
:100A1000BF92CF92DF92EF92FF920F931F93CF93EB
:100A2000DF93CDB7DEB7CA1BDB0B0FB6F894DEBF82
:100A30000FBECDBF09942A88398848885F846E84A8
:100A40007D848C849B84AA84B984C884DF80EE80F2
:100A5000FD800C811B81AA81B981CE0FD11D0FB6FB
:100A6000F894DEBF0FBECDBFED010895F894FFCF1F
:100A70000100010202030303030404040404040448
:100A80000405050505050505050505050505050517
:100A900005060606060606060606060606060606F7
:100AA00006060606060606060606060606060606E6
:100AB00006070707070707070707070707070707C7
:100AC00007070707070707070707070707070707B6
:100AD00007070707070707070707070707070707A6
:100AE0000707070707070707070707070707070796
:100AF0000708080808080808080808080808080877
:100B00000808080808080808080808080808080865
:100B10000808080808080808080808080808080855
:100B20000808080808080808080808080808080845
:100B30000808080808080808080808080808080835
:100B40000808080808080808080808080808080825
:100B50000808080808080808080808080808080815
:100B60000808080808080808080808080808080805
:020B700008007B
:00000001FF
